:100000006AC40000A0C400009EC400009CC400009C
:100010009AC4000098C4000096C4000094C4000074
:1000200092C4000090C400000C949D2D0C94ED2E01
:100030000C94522D88C4000086C4000084C40000C3
:1000400082C4000080C400007EC400007CC40000A4
:100050000C94E02C0C94792D76C4000074C400003C
:1000600072C4000070C400006EC400006CC40000C4
:100070006AC4000068C4000066C4000064C40000D4
:1000800062C4000060C400005EC400005CC40000E4
:100090005AC4000058C4000056C4000054C40000F4
:1000A00052C4000050C400004EC400000631FF09D5
:1000B00074A1010975150026FF00952075088102BD
:1000C000C005010902A10185020901A10005091964
:1000D000012908150025019508750181020501090E
:1000E0003009311581257F9502750881060938157B
:1000F00081257F950175088106050C0A3802158156
:10010000257F950175088106C0C005010980A10100
:10011000850319012AB700150126B700950175104E
:100120008100C0050C0901A101850419012AA00262
:10013000150126A002950175108100C00660FF0917
:1001400061A1010962150026FF0095207508810252
:100150000963150026FF00952075089102C005016E
:100160000906A101050719E029E7150025019508F1
:10017000750181029501750881010507190029FFA4
:10018000150026FF0095067508810005081901294C
:1001900005150025019505750191029501750391DD
:1001A00001C000000000000000000000000000008E
:1001B000000000000000000000000000000000003F
:1001C0000000000000007E0F00D4FFFFFFC700000A
:1001D000007800000000000000002A2B280000002A
:1001E00000000000000000000000000000290000E6
:1001F00000002C1E3420212224342627252E362DC3
:100200003738271E1F202122232425263333362E5C
:1002100037381F0405060708090A0B0C0D0E0F10CE
:100220001112131415161718191A1B1C1D2F313013
:10023000232D350405060708090A0B0C0D0E0F10B7
:100240001112131415161718191A1B1C1D2F3130F3
:10025000354C09027400040100A0FA0904000001F1
:100260000301010009211101000122440007058159
:100270000308000109040100020300000009211124
:100280000100012222000705820320000107050367
:1002900003200001090402000103000000092111EC
:1002A000010001227B0007058403200001090403EB
:1002B00000010300000009211101000122150007BF
:1002C0000585032000011201000200000008646996
:1002D00075000100010203011C0376006900610042
:1002E0006C003A00660036003400630032006200A1
:1002F0003300630000000A03490044003700350062
:1003000000000E03490044004F00420041004F002E
:100310000000040309045B435D005B445D005B5324
:100320005D005B575D005B525D00290A002575008A
:100330002F002575005D280025640020002564003D
:10034000200025640020002564007C002530325800
:10035000006D6F7573656B6579205B62746E7C7878
:100360002079207620685D287265702F61636C2982
:100370003A205B0029001E001F00200021002200FF
:100380004C00230024002500260027002D002E000D
:100390004600350014001A000800150017002A0056
:1003A0001C0018000C00120013002F003000390050
:1003B0002B0004001600070009000A0028000B00AB
:1003C0000D000E000F003300340031004B00E1003F
:1003D0001D001B0006001900050028001100100078
:1003E000360037003800E50052004E00E0000405FA
:1003F000E300E20021522C002C002C006152E600A8
:10040000E4000F08500051004F00007C3A003B0010
:100410003C003D003E0000003F0040004100420023
:10042000430044004500A500037CBD0025782778E3
:10043000237829782178D900D100CD00D200D900C5
:100440000000A600A700027CBE0026782878247849
:100450002A782278DA00CF00CE00D000DA0000003F
:1004600000004A0001000000000000000000000041
:10047000207800000000000000000000A800A90093
:100480004D0001000000010001000100000000001B
:100490000000010001000100AE00AC00AA00AB00AA
:1004A0000100010001000100010001000100010044
:1004B0000100010001000100010001000100010034
:1004C0000100010001000100010001000100010024
:1004D0000100010001000100010001000100010014
:1004E0000100010001000100010001000100010004
:1004F00001000100010001000100010001000100F4
:1005000001000100010001000100010001000100E3
:1005100001000100010001000100010001000100D3
:1005200001000100010001000100010001000100C3
:1005300001000100010001000100010001000100B3
:1005400001000100010001000100010001000100A3
:100550000100010001000100010001000100010093
:100560000100010001000100010001000100010083
:100570000100010001000100010001000100010073
:100580000100010001000100010001000100010063
:100590000100010001000100010001000100010053
:1005A0000100010001000100010001000100010043
:1005B0000100010001000100010001000100010033
:1005C0000100010001000100010001000000000025
:1005D0000000000000000001010203040506080AF3
:1005E0000C0F1114181C2024292E33393F464C536C
:1005F0005B626A7179818A929AA2AAB2B9C1C8CFA4
:10060000D5DCE1E7EBF0F4F7FAFCFDFEFFFEFDFCC4
:10061000FAF7F4F0EBE7E1DCD5CFC8C1B9B2AAA292
:100620009A928A8179716A625B534C463F39332EC4
:100630002924201C1814110F0C0A080605040302B3
:1006400001010000000000000000000000010101A5
:10065000010101010101020202020202020202037F
:10066000030303030303030404040404040405054F
:100670000505050606060606070707070708080812
:1006800008090909090A0A0A0B0B0B0C0C0C0D0DC1
:100690000D0E0E0E0F0F0F10101111111212131359
:1006A0001414151516161717181819191A1A1B1BD2
:1006B0001C1D1D1E1E1F202021222223242425262E
:1006C00026272829292A2B2C2D2D2E2F3031323266
:1006D000333435363738393A3B3C3D3E3F40414272
:1006E000434445464748494A4C4D4E4F5051535458
:1006F000555658595A5B5D5E5F616264656668690C
:100700006B6C6D6F7072737577787A7B7D7E80828B
:10071000838587888A8C8E8F91939596989A9C9ED4
:10072000A0A2A3A5A7A9ABADAFB1B3B5B7BABCBEE4
:10073000C0C2C4C6C9CBCDCFD1D4D6D8DBDDDFE2B1
:10074000E4E7E9EBEEF0F3F5F8FAFDFF0A002530F7
:10075000313662003A200025303258000A722F6389
:10076000203031323334353637383941424344450D
:10077000460A00643214783C1EFD377A585A00004D
:1007800004E6D6B4460200210116000000742FE5ED
:10079000A3E0027500EA5D003D8889C65436C317A0
:1007A0004FE4E04BA1DB7A6EB4D0C1E4A041996E76
:1007B0000211E74DF2CD31985523B102D8EBB46860
:1007C0009F8FD885311D049C91691A741F12190BD3
:1007D000BA49B1869D4527E9344742D123070D9890
:1007E000CF7BA6F0DE687D94D175E0599864203106
:1007F000D0D94CC4BD513F418C79B37BF0A66294F3
:10080000D5EA0A86931CEED63740F4280AD1506305
:10081000AD579988D730A591DCF213C087D9EE285F
:100820009D5CFDFE101D2F8EA891AE71B7586C9A7D
:100830001E48E92E40DA9681E13C0E317F14C672E3
:10084000CFF425900EF097B6E24540BE80394202C3
:10085000627D47768D876F3AFDB0B2E19F7CE49B65
:1008600079A4B07D9DB7982079E8A7D7128CA764AA
:1008700003FAEF47A514270246F3F2D37E0FCBF518
:10088000C2150000009E91A9A31FB8FA18000186A6
:1008900002F6040000DF9178D5B1C467FB020000C6
:1008A000000004595A504F52514A4D4B4E2A4C2F7A
:1008B00030B6B7ABACBBBCA9AABDBECFD0CDCEDBEA
:1008C000DCD9DA0D0E0B0F1A0508050905071811FA
:1008D000130408120C0011241FBECFEFDAE0DEBFB4
:1008E000CDBF04B603FE18C0809114049091150486
:1008F000A0911604B09117048730904BA740B04BDD
:1009000059F41092140410921504109216041092C7
:100910001704E0E0F8E3099511E0A0E0B1E0E4E5B8
:10092000F2E602C005900D92AC3BB107D9F724E086
:10093000ACEBB1E001C01D92A431B207E1F70E9417
:100940008E240C94CF305CCBFF93EF93E091BC01ED
:10095000F091BD01309709F00995EF91FF9108954D
:10096000FC018591803011F0EFDFFBCF0895FF2768
:10097000E0E230E247FF0CC0419597FF09C0EDE28D
:100980006095709580959095611D711D811D911DDB
:1009900027FF02C0219530E350E2AA27660F771F98
:1009A000881F991FAA1FA41710F0A41B63955A95BE
:1009B000A9F7AA3008F0A95FA05DAF93F395611580
:1009C00071058105910541F7ED3211F4EF93F3952F
:1009D000F21718F43F93F395FBCF8F91B5DFFA959B
:1009E000E1F70895E991F9918591803021F0853200
:1009F00019F0AADFF9CF089520E0E8945591553217
:100A0000C1F3503311F4689455915A3348F450535C
:100A100090F3220F022E220F220F200D250FF4CF6C
:100A20000EF4219589919991533619F3533729F191
:100A3000533559F1BC0188279927E8945C3621F495
:100A40008991999168945591543639F446EF7EF026
:100A500077FF0DC08FEF9FEF0AC055374AE039F09E
:100A6000583540E121F0523642E009F00895FF93F5
:100A7000EF937DDFEF91FF91B7CFFF93EF93FC01F1
:100A800081918030B9F360DFFBCFFF93EF9368DF94
:100A9000F1CFDF93CF93CDB7DEB72596A3DFCF910C
:100AA000DF9108959C019A9581159F4118F5F32FC8
:100AB000F270EE27832F8170732F74706627532F87
:100AC0005870442734FF0CC08295807FEF2B09F0CB
:100AD0008062672B09F08064452B69F08068089577
:100AE000EF2B09F08260672B09F08460452B19F029
:100AF0008860089580E00895CF93DF93EB01D2DF03
:100B0000FE010995DF91CF9108950C94D92F089596
:100B1000982F92959F7024E0911102C020E0982FA9
:100B2000892F86958695811511F02E5F982F892F34
:100B30008695820F08958295982F990F990F9C7C26
:100B4000869586958373982B892F880F8A7A969538
:100B50009575892B0895809310040895809311044E
:100B6000089521E030E001C0220F8A95EAF78091D4
:100B70001104822BF3CF21E030E0A90102C0440F21
:100B8000551F8A95E2F7CA01809590911104892337
:100B9000E5CF292F953090F58F3080F590E03FE03C
:100BA000239F800D911D1124282F277041E001C043
:100BB000440F2A95EAF723E0969587952A95E1F761
:100BC000FC01EE0FFF1FE80FF91FEF58FD4F20E06B
:100BD00030E070E05191DF01CB01022E02C096950A
:100BE00087950A94E2F7817081958527842385276C
:100BF0008E932F5F3F4F2330310561F70895292FE2
:100C0000953078F58F3068F590E03FE0239F800DB8
:100C1000911D1124682F677023E0969587952A957A
:100C2000E1F7FC01EE0FFF1FE80FF91FEF58FD4F32
:100C300040E050E080E0219130E0062E02C0369581
:100C400027950A94E2F721703327042E01C0220F62
:100C50000A94EAF7822B4F5F5F4F4330510559F7F3
:100C6000089580E008959091110421E030E0F901A9
:100C700001C0EE0F8A95EAF7D90102C0AA0FBB1F87
:100C80006A95E2F7EA2B01C0220F4A95EAF7892F0D
:100C90008E23E81303C0892F822B60CF2095822FEB
:100CA0008923FBCF982F90958091130489238093FB
:100CB00013040895803E9105D9F1C8F4813391055C
:100CC00009F482C048F48932910509F472C08A326D
:100CD000910509F480C0089589339105E9F08238BF
:100CE0009105D1F08533910509F45EC00895843EE5
:100CF0009105D9F148F4823E910539F1833E910581
:100D000049F181EE90E00895863E9105C9F1873E54
:100D1000910509F43EC0089520915F0223702111CE
:100D200064C02091600223FF14C089E290E008951E
:100D300020915F0220FD45C03091600230FF09C064
:100D400024FD24C083EE90E0089520915F0222FDEF
:100D5000F7CF089520915F0222FD44C030916002D8
:100D600030FD43C024FFF5CF11C02091600221FF68
:100D7000F0CF80915F0284FD09C087EE90E0089576
:100D800020915F0223FFE5CF24FFF7CF80E090E0C2
:100D9000089520915F0223FD2BC03091600231FF46
:100DA000E1CF84EE90E0089520915F0225FFD1CF3E
:100DB000BCCF20915F0225FD1EC02091600223FF61
:100DC000C8CF89E390E0089520915F0226FFC1CF4C
:100DD0008AE290E0089520915F0226FFBACF81E376
:100DE00090E0089582EE90E0089580EE90E00895FE
:100DF00086EE90E0089585E390E0089590915F027B
:100E000092FF10C041E0282F2471243009F040E007
:100E100031E0282F2871283009F030E0431711F015
:100E20002CE0822793FF10C041E0282F2471243149
:100E300009F040E031E0282F2871283109F030E036
:100E4000431711F02CE082273091600230FF10C070
:100E500051E0282F2171213009F050E041E0282F86
:100E60002871283009F040E0541711F029E082275A
:100E700031FF10C041E0282F2171213109F040E0FD
:100E800031E0282F2871283109F030E0431711F0A4
:100E900029E0822794FD877E08951F93CF93DF93E7
:100EA00009DFEC01811520E59207D8F5811540E2B4
:100EB000940708F0E2C0833C9105C0F4883A91059C
:100EC00008F098C0853A910570F4049738F481E0F1
:100ED000219709F080E0C82F50E0D52FCE01DF9197
:100EE000CF911F910895A497D064F8CF883E9105C3
:100EF00058F4803E910590F78D5C9109D065439739
:100F000068F3C0E0D0E0EACF9A9581159F41C8F719
:100F10008D2F74DF182FCE019927CCDEEC01D12B59
:100F2000DDCFC03682E5D80738F5C03492E5D90761
:100F300008F07FC0C03222E5D207B8F48C2FC1156B
:100F400042E5D40708F061C08F7158DF63E0CC0F31
:100F5000DD1F6A95E1F7CC27DF70282F30E084FD94
:100F600086C0C22BD32BD069B9CFCF71D0E0DC2F94
:100F7000CC27C16FD06AB2CFC03C52E5D50708F587
:100F8000C03A62E5D60708F06AC0CE0180569245A5
:100F9000809708F0B6CF8C2F86958695877050E2A3
:100FA000859FC0011124C37021E030E0A90102C077
:100FB000440F551FCA95E2F7EA01C82BD92BDA680E
:100FC0008DCFCE01805C9245809708F09ACFCE01FC
:100FD00023E0880F991F2A95E1F7807E9927C37037
:100FE000DD2721E030E0A90102C0440F551FCA955A
:100FF000E2F7E2CFC85AD0E0CC0FDD1FC15BDE4F75
:101000000990D881C02DD46469CF8695869520E259
:10101000829FC0011124C37021E030E0A90102C009
:10102000440F551FCA95E2F7EA01C82BD92BDD689A
:1010300055CF8C2F86958695877050E2859FC0018D
:101040001124C37021E030E0A90102C0440F551FF4
:10105000CA95E2F7EA01C82BD92BDC683FCF8C2F69
:101060008F71CCDEC82FD0E0DC2FCC2737CF90E1BA
:10107000899F90011124332774CF99271BDEEC013F
:101080002DCFF894E82FE295EF70F0E041A18F703A
:1010900021E030E0B90102C0660F771F8A95E2F7C0
:1010A000CB01962F9095942391A392A1892B82A393
:1010B000789408950895CF92DF92EF92FF921F9354
:1010C000CF93DF93172FE82FF0E0E45BF94F711116
:1010D0000CC0E4918E2F7E2F6E2FDF91CF911F9148
:1010E000FF90EF90DF90CF900895E62EF12CC72E61
:1010F000D12CF491EF2F86E0689F90011124CFEF5F
:10110000D0E0C901BE010E948A2FAB01EE0CFF1C8A
:1011100065E5649FC001659F900D1124E81AF90AE6
:101120006E2D660F6E0D7E01EC18FD08FE9DD00140
:10113000FF9DB00D11248B2F169F70011124EF2CF1
:10114000FF246E01CE18DF087601FE9D6001FF9D31
:10115000D00C11247E01E61AF108B701169F700128
:10116000179FF00C1124EF2CFF24CE19DF09FC9FF0
:101170007001FD9FF00C11247F2D43305105C1F00B
:101180002C3F334058F441305105B1F04230510505
:1011900009F0A2CFEB2F8F2D7F2F9ECF443051052A
:1011A00071F04630510509F497CF7B2F8D2D94CFE8
:1011B0007D2DEB2F8F2F90CF7F2FED2D8DCFEF2D0E
:1011C0007B2FF8CF80910704843028F483708460EB
:1011D0008093070408958C32E8F383708862F8CF17
:1011E000CF93DF938091070480FD0BC0C0E0D0E077
:1011F00020E040E060E0CE017CD12196C031D105F5
:10120000B9F7DED4DF91CF910895FF920F931F932A
:10121000CF93DF93182F062FF42E8091070480FFC1
:101220000CC0C0E0D0E02F2D402F612FCE0161D146
:101230002196C031D105B9F7D3DFCDB7DEB7E5E0F0
:101240000C94612FCF93DF93EC018091070480FF12
:101250000BC0709109046C8180910A042CDF962FD9
:10126000672F482F892FD1DF8C818F5F8C83DF918F
:10127000CF910895FF920F931F93CF93DF93EC01CB
:10128000F12C00E010E0709109046C816F0D8091E9
:101290000A0411DF472F282FC8012BD10F5F1F4FE2
:1012A0008FE0F80E0031110571F79ADF8C819A8179
:1012B00090FF07C08F5F8C83CDB7DEB7E5E00C945D
:1012C000612F8150F8CFA0E0B0E0E9E6F9E00C949E
:1012D0003E2F8C0180918600909187006CE070E039
:1012E0000E948A2F6017710768F0C80169E070E0FA
:1012F0000E948A2F262F972F822FCDB7DEB7ECE0E2
:101300000C945A2F8091860090918700E09086007F
:10131000F0908700C0908600D0908700C6E0D0E0B3
:10132000BE010E948A2F20E030E0060F171F211D0A
:10133000311D4801590185E0880C991CAA1CBB1C71
:101340008A95D1F7C701BE010E948A2FE12CF12CAA
:10135000A7019601260F371F411D511DC501B4017C
:101360000E94B12F69017A01E0918600F091870017
:10137000CA01B9010E946F2F9B01AC01DF010E94DD
:10138000FF2F9B01AC01C701B6010E946F2FDC014A
:10139000CB012FE0B695A795979587952A95D1F71C
:1013A0002091860030918700281739071A061B06FE
:1013B00020F48091860090918700282F9DCF843063
:1013C000E0F481111BC090918000977F9093800082
:1013D0002091860030918700A82FB0E00E94F02F66
:1013E00023E030E040E050E00E94B12FC9016BDF04
:1013F00090938D0080938C00089583E090918000FD
:101400009860E4CF982F990F990F990F2091FF02C0
:101410002770922B9093FF0221E0983008F420E08F
:101420009091FF0220FB90F99093FF02C8CF8115A5
:101430002CE7920741F420915C0230915D02232B4E
:1014400011F480E090E00895E9E8F3E080E090E0B6
:101450006AE572E24DE752E22FEE32E2768365836F
:1014600050874783328721879687858701963F96E5
:101470008830910599F70895FB01811520E29207C4
:1014800028F4811541E0940738F408959C01305206
:101490002115304348F00895392F94FF02C032954A
:1014A000307F2081232B208399270895462B22FF0C
:1014B0000FC0982F92959F708F70892B962F9295C1
:1014C0009F706F70692B942F92959F704F70492B6E
:1014D000982F9623961309C050E04095509590E0C0
:1014E0004823592381E0452B09F080E00895809A34
:1014F0000895FC01EE0FFF1FE80FF91FE951FE4FA1
:101500006183408322830895FC01848186238111B5
:101510000AC082818115B9F06823908593FF05C0C8
:1015200081E061110FC080E00895282F22952F706F
:101530008F70282B962F92959F706F70962B81E05D
:101540002913F1CF089581E008950F931F93CF934E
:1015500001E010E0082E01C0000F0A94EAF7C091E4
:101560000F049C2F9023911108C0FBDAC027C09371
:101570000F04CF911F910F910895FDDAF7CF282F17
:1015800035EB2303C001112497FF04C08058910953
:10159000892F089580589F4FFBCF8091910280FD45
:1015A00014C081FD14C082FD16C080919002811587
:1015B00081F08E3180F420E5829FC00111246EE11C
:1015C00070E00E949E2F862F089584E1089588E29E
:1015D000089588E0089580E508958091910280FD46
:1015E00017C081FD17C082FD19C080918F0281153F
:1015F00099F0883298F428E0829FC001112468E2B3
:1016000070E00E949E2F6115710551F0862F08959C
:1016100062E0FCCF64E0FACF61E0F8CF68E0F6CF9B
:1016200081E008959091EB0289029001112437FF27
:1016300003C08093EB0208952F3731051CF4980FF7
:101640009093EB0208959C0180E090E0F901E80F8F
:10165000F91FE491E41307C091E08927F901E80F2D
:10166000F11D849108950196861780F380E0089516
:10167000FA01309709F009950895E0916702F09119
:101680006802309739F00190F081E02D309711F029
:101690000995089580E00895A3E0B0E0E2E5FBE05D
:1016A0000C94482F9C018091E5019091E6018217EE
:1016B0009307B1F03093E6012093E501E0916702D2
:1016C000F0916802309761F00084F185E02D309749
:1016D00039F083E089833B832A83CE010196099503
:1016E0002396E2E00C94642FA3E0B0E0EAE7FBE08D
:1016F0000C94482F9C018091E3019091E4018217A2
:101700009307B1F03093E4012093E301E091670285
:10171000F0916802309761F00084F185E02D3097F8
:1017200039F084E089833B832A83CE0101960995B1
:101730002396E2E00C94642F9C01FC0132968FEF1B
:1017400090E04191461751F08F3F19F4411101C0CB
:10175000892F9F5F9630A9F78F3F09F40895280FCE
:10176000311D87FD3A95F90162830895E0ECF1E0BF
:101770009191891302C0DF011E9291E0E63CF907C6
:10178000B9F708958091030108952FB7F8948091D7
:10179000DF019091E001A091E101B091E2012FBF42
:1017A00008952FB7F8946091DF017091E001809166
:1017B000E1019091E2012FBF0895CF92DF92EF9265
:1017C000FF92CF93DF93D82FC92FC0908303D0907F
:1017D0008403E0908503F0908603E3DF6C197D09B4
:1017E0008E099F09643F71408105910510F1D9DF91
:1017F0006B017C0182E390E0A0E0B0E0C0923F0288
:10180000D0924002E0924102F092420280933B0269
:1018100090933C02A0933D02B0933E02D09381038B
:10182000C0938203DF91CF91FF90EF90DF90CF9034
:10183000089584EF91E0A0E0B0E0E0CF0895FC01CE
:101840009B018091D3019091D4018617970740F0B6
:10185000672B29F48091E8008E778093E800C90116
:1018600040E0009741F4411106C08091E80082FFFA
:101870002FC080E0089520915E022115A9F1253046
:10188000A9F12091E80023FD2DC02091E80022FD60
:10189000ECCF2091E80020FFE4CF3091F3002091BD
:1018A000F200009719F02830310558F041E0283057
:1018B000310509F040E02091E8002E772093E80000
:1018C000D0CF41914093F10001972F5F3F4FE9CF77
:1018D00080915E02811541F0853041F08091E800F1
:1018E00083FFC3CF81E0089582E0089583E00895E7
:1018F0008091CD0187FF13C08091E80082FF06C070
:101900008091E8008B778093E800089580915E02D3
:101910008111F2CF089580915E028115D9F38091F3
:10192000E80080FFF8CF8091E8008E77ECCF20911F
:10193000E4003091E50095E6A9012091EC00822FAA
:10194000817020FF06C08091E80080FF06C080E023
:1019500008952091E80022FD1AC080915E02811551
:1019600089F0853089F08091EB0085FD0FC02091D2
:10197000E4003091E50042175307F9F29A95E1F639
:1019800084E0089582E0089583E0089581E0089559
:10199000E8EDF0E080818E7F80831092E20010926B
:1019A000DA001092E100A0EEB0E08C9181608C939F
:1019B00080818F77808319BCA7EDB0E08C918E7FFA
:1019C0008C9380818F7E80831092CC010895E0916A
:1019D0006702F0916802309739F00284F385E02DB8
:1019E000309711F060E209950895982F9093E900DF
:1019F000891771F07091EC002091ED005091F0008A
:101A000021FD09C09F5F973089F78093E900089511
:101A1000762F242F50E03091EB003E7F3093EB0087
:101A20003091ED003D7F3093ED003091EB0031605F
:101A30003093EB007093EC002093ED005093F00096
:101A40002091EE0027FDDECF0895A0E0B0E0EBE2AC
:101A5000FDE00C94422FC8EDD0E088818F7E888312
:101A6000E7EDF0E080818160808384E082BF81E0E7
:101A70008093CC0188818E7F888302EE10E0F8018C
:101A800010821092DA0081EEC82ED12CF60110825D
:101A900088818F77888388818068888388818F7D1B
:101AA000888319BC10925E021092CB0110922F0213
:101AB0001092CA0190EEE92EF12CF70180818B7F04
:101AC000808388818160888342E060E080E08DDFF0
:101AD000F60180818E7F8083F80180818160808320
:101AE000808188608083F70180818E7F80838881F8
:101AF00080618883CDB7DEB7E8E00C945E2F9FB796
:101B0000F8941092D6019FBF90915E02943009F034
:101B100047C02091E9009091EC002F70979599278C
:101B20009795922B25E02093E9002091EB0020FF70
:101B300034C02091EE0027FF30C02091D50121153F
:101B400021F02091E80025FF28C01092D50126E061
:101B50003091E80035FF14C08093F1008091E800D7
:101B600085FD27C08091E80080FFFCCF8091E800D0
:101B70008E778093E8009F709093E90080E008954D
:101B800030915E02343049F43091EB0035FD05C0F0
:101B90002A9541F481E08093D5019F709093E900EC
:101BA0008FEF0895EFE9FFE03197F1F700C00000F3
:101BB000CFCF8FB7F89421E02093D6018FBFDBCF32
:101BC00031B33E7F21B321604FB7F89487EE91E0A7
:101BD000FC010196508168E021BB000000C057FF66
:101BE00031BB550F000000C000C000C031BB00C0B9
:101BF0006A9591F752E08731950751F74FBF8FE50E
:101C000094E00197F1F700C00000089581E080930F
:101C1000E00080E28093D8001092C9008FE19EE43A
:101C20000197F1F700C0000087E090EBDC018093A2
:101C3000140490931504A0931604B093170488E13C
:101C40009CE00FB6F894A895809360000FBE909327
:101C50006000FFCF0F931F93CF93DF938B01EA01B7
:101C600090915E02943051F58093E9008FEF90914E
:101C7000E80095FD06C095ED9A95F1F700008A956C
:101C8000B1F78091E80085FF19C051DE811111C0C4
:101C90008091E80085FD06C08091E8008E778093F2
:101CA000E800F3CFF80181918F018093F100219733
:101CB00079F78091E8008E778093E800DF91CF91EB
:101CC0001F910F910895792F603229F440E250E07E
:101CD000682F82E0BFCF0895CF93DF93D82FC92F0D
:101CE00048E050E0682F792F81E0B4DF88E0ED2FE5
:101CF000FC2FA7EDB1E001900D928A95E1F7DF91FD
:101D0000CF910895BC0146E050E084E0A3CFBC0130
:101D100043E050E084E09ECFFC01608186E090E0EB
:101D20000C949A308091FF0281FD11C082608093F3
:101D3000FF028FEF92E0F0DF10922C0210922B0244
:101D400010922A0280916F00816080936F00089545
:101D50008091FF0281FF11C08D7F8093FF028FEF82
:101D600092E0DADF80916F008E7F80936F00809128
:101D7000FF0286958695869522CB08951F93CF9373
:101D8000DF93962F122F632F8430D8F49530C8F448
:101D90004F30B8F4C42FD0E0CC0FDD1F2EE1929F5E
:101DA000C00DD11D112496E9899FC00DD11D1124AC
:101DB000CE0189960E949A30612FCE018A960E94A8
:101DC0009A30DF91CF911F910895909113048091E3
:101DD0001204982B80910503809589239091040328
:101DE000892B8093BE0148E050E069E672E08EEBFB
:101DF00091E00E945530892BB9F088E0EEEBF1E0DC
:101E0000A9E6B2E001900D928A95E1F7E0916702B0
:101E1000F0916802309741F00280F381E02D309715
:101E200019F08EEB91E009950895811531F09091AC
:101E30001304892B80931304C8CF0895811519F0DA
:101E40000E945206C2CF0895811531F0909112047C
:101E5000892B80931204B9CF0895811539F08095AC
:101E600090911204892380931204AFCF089580913A
:101E70000003811521F082E2F0DF10920003089543
:101E8000CF93DF93EC0149855A856D857E85F0DB24
:101E90009B8190958091120489238093120495DF91
:101EA00085E0FE0111928A95E9F7DF91CF910895BF
:101EB000CF93DF93EC018C8181FD0FC082608C8316
:101EC000809112049B81892B809312047EDF4F81C5
:101ED00058856D857E85CE01CBDB10920204109271
:101EE00001048C8180FD02C0CE01CADFDF91CF9159
:101EF000089586E090E00E9479308093FF0282FD91
:101F000006C08DE18093FF028FEF92E005DF8091A4
:101F1000FF02803220F0877088618093FF029091E9
:101F2000FF02892F817090FF04C0892F86958695C6
:101F3000869545CA0F931F93CF93DF93843030F576
:101F4000653020F54F3010F5C42FD0E0CC0FDD1FE9
:101F50002EE1629FC00DD11D112436E9839FC00D73
:101F6000D11D1124CE0189960E947930082F10E0EE
:101F7000102F0027CE018A960E9479309801282BD5
:101F8000C901DF91CF911F910F91089580E090E0FA
:101F9000F8CF462F672F2091630230916402232BE4
:101FA00081F4703F39F4403F61F480916102909177
:101FB00062020895753028F44F3018F4843008F424
:101FC000B9CF80E090E00895A0E0B0E0EAEEFFE055
:101FD0000C94432F7C010091110480911004082B74
:101FE000C3E0D0E010E0C8010C2E02C095958795A3
:101FF0000A94E2F780FD09C02197A8F7D12C8D2D16
:10200000CDB7DEB7E7E00C945F2FDC2EB7018C2F45
:10201000C0DF0E944D07019779F3F1CF0F931F9313
:10202000CF93FC0186819781009789F48581008197
:102030001181811581F0611571F0C801C5DFC82FCC
:10204000682FC8010E94C905B8018C2FA2DFCF916B
:102050001F910F910895C8010E94FF05C82FF4CF6A
:10206000382F292FCB01A32FB22F8F3A9105A1052D
:10207000B10520F48F5A9C4F0C94793080E008957C
:1020800085E290E00E9479308A3889F486E290E017
:102090000E947930833E59F487E290E00E947930C3
:1020A00091E0823209F090E0892F8170089580E0FC
:1020B000FCCFAAE0B0E0EFE5F0E10C943D2FC0903A
:1020C0005C02D0905D0281E090E090935D0280938D
:1020D0005C02812C912CE12C5401F12C14C0F801EC
:1020E00025913591472D6F2D8E2D48DE0E5F1F4FA8
:1020F00073948FE07812F3CF9FE0A90EB11CF39494
:10210000E5E0FE1639F08501000F111F0C581C4F39
:10211000712CE5CFE394FBE48F0E911C84E0E81270
:10212000DBCF1A8219821C821B821E821D821886B6
:102130001F8288EC90E09A87898701E812E0FE010F
:1021400031967F014AE050E0B801C7010E94B830E3
:10215000065F1F4F013DF2E01F07A1F789E0F7017D
:1021600011928A95E9F78FEF9FEF9E838D8387E029
:102170008A874AE050E0B801C7010E94B830065F84
:102180001F4F0132F3E01F07A1F786E0F70111921C
:102190008A95E9F746E050E0B801C7010E94B830DF
:1021A0000A5F1F4F0135F3E01F07A1F7D0925D02D0
:1021B000C0925C022A96EDE00C94592FAAE0B0E0A0
:1021C000E4EEF0E10C94402F06E013E081EDE82E00
:1021D00082E0F82E97E0B92E27E1C22E22E0D22E1F
:1021E000AA24A3944AE050E0B701CE0101960E94D0
:1021F0006930F8013896DF018B2D1D928A95E9F739
:1022000089819A81D80111969C938E938F81129621
:102210008C9312978D8113968C93139788851496BF
:102220008C931497898515968C9315978B819C8137
:1022300017969C938E9316978A8587FD04C01E96E9
:10224000DC92CE921D9780FF02C0F801A08681FF2C
:1022500007C0D80118969C911897926018969C9385
:1022600082FF04C0F80190859460908783FF07C0C7
:10227000D80118969C911897986018969C9384FFA3
:1022800004C0F80190859061908785FF07C0D80150
:1022900018968C911897806218968C93BAE0EB0E82
:1022A000F11C015F1F4FE1E2EE16E3E0FE0609F0CC
:1022B00099CF2A96EAE00C945C2FA6E0B0E0E3E622
:1022C000F1E10C94432F01EA12E081E2E82E83E071
:1022D000F82E98E0D92E46E050E0B701CE010196E5
:1022E0000E946930F8018D2D11928A95E9F7B801A5
:1022F0006C5F7F4F89819A81BFD8F8019183808379
:10230000B8016B5F7F4F8B819C81B6D8F8019383B6
:1023100082838D8186838E818783F6E0EF0EF11CA8
:10232000085F1F4F81E5E81683E0F806A1F62696C0
:10233000E7E00C945F2F282FCB01283070F44AE09F
:10234000249F90011124B9016F577D4F4AE050E05E
:102350000E94693080E090E008958FEF9FEF08952C
:102360008091300283FF96C081E593E09F938F9325
:102370000E944905809193021F928F938CE493E011
:102380009F938F930E9449058AE493E09F938F93D4
:102390000E94490580919402282F082E000C330BCF
:1023A0003F938F9387E493E09F938F930E94490517
:1023B00085E493E09F938F930E9449058091950255
:1023C000282F082E000C330B3F938F9382E493E069
:1023D0009F938F930E94490580E493E09F938F938E
:1023E0000E94490580919602282F082E000C330B7D
:1023F0003F938F938DE393E09F938F930E944905C2
:102400008BE393E09F938F930E94490580919702FD
:10241000282F082E000C330B3F938F9388E393E013
:102420009F938F930E94490585E393E09F938F9339
:102430000E9449058DB79EB780960FB6F8949EBF4F
:102440000FBE8DBF809190021F928F9382E393E025
:102450009F938F930E94490580E393E09F938F930E
:102460000E944905809191021F928F938DE293E023
:102470009F938F930E9449058AE293E09F938F93E5
:102480000E9449058DB79EB70C960FB6F8949EBF73
:102490000FBE8DBF7AD92091940230919502232BE3
:1024A000211521F080934B0290934C0220919602CB
:1024B00030919702232B211521F0809349029093AC
:1024C0004A02E0916702F0916802309759F0068065
:1024D000F781E02D309731F082E08093920282E91B
:1024E00092E009950895611509F441C0E3E3E80F0E
:1024F000E33148F4F0E0EF52FF4C0C94D32F4DD869
:102500008195809395022CCF48D8FBCF46D88195F2
:1025100080939402F8CF41D8FBCF5FD88093960286
:10252000F2CF5BD88195FACF58D8819580939702E6
:10253000EACF53D8FBCF815D990B21E030E001C099
:10254000220F8A95EAF780919302822B809393025F
:10255000DACF80919102816080939102D4CF8091F3
:1025600091028260F9CF809191028460F5CF409111
:1025700094028D3C59F48091950287FF0DC0109212
:102580009502411559F41092900208C08E3C81F4D6
:102590008091950218169CF3411581F08091960266
:1025A00090919702892B8111AECF10928F02ABCF01
:1025B0008F3C41F447FFF0CF109294028091950236
:1025C0008115E0CF803D19F41416B4F3E5CF909156
:1025D0009602893D29F41916FCF610929602DCCF7A
:1025E0008A3D19F497FFD8CFF8CF909197028B3D91
:1025F00029F497FFD1CF10929702CECF8C3D19F4DA
:102600001916CCF3C9CF9FE2980F983090F4815DF2
:10261000990B21E030E0B90102C0660F771F8A955F
:10262000E2F7CB01809590919302892380939302E6
:10263000B3CF8D3D31F4809191028E7F80939102D2
:10264000ABCF8E3D21F4809191028D7FF7CF8F3DEE
:1026500009F0A2CF809191028B7FF0CFCF93C82F4A
:102660008115A1F08CEF8C0F813A90F4E0ECF1E051
:1026700086EC91E02191C21709F43BC08E179F07A9
:10268000C9F76C2F8EEB91E057D89FDBCF9108955F
:1026900080E28C0F883068F4C77021E030E001C020
:1026A000220FCA95EAF780911304822B80931304BA
:1026B000ECCF8BE58C0F833038F42C2F2452330B66
:1026C000C9010E944C0BE2CFE8E5EC0FEB3148F476
:1026D000F0E0EE0FFF1FEB57FE4F8081918104D891
:1026E000D5CF83E38C0F833188F661E08C2FFBDE3E
:1026F000CDCF8C2F3BD869DBC4CFCF93DF93EC01D8
:10270000805E9109089720F064E27FE0209711F441
:1027100065E17FE0CE010E947C058C2F9FDFDF9179
:10272000CF910895811551F19CEF980F913A10F4D3
:102730001DD84BCB90E2980F983050F4877091E001
:1027400001C0990F8A95EAF7892F0E945206F1CFAE
:102750009BE5980F933020F480E090E00C944C0BB4
:1027600098E5980F9B3120F480E090E00C94740B76
:1027700093E3980F933110F460E0B5CE08951F9362
:10278000CF93DF93182FEB0169DF209731F4812F6E
:10279000C9DFDF91CF911F9108958FE99FE00197E5
:1027A000F1F700C000002197F0CFA0E0B0E0EBED22
:1027B000F3E10C94412FEC018881811509F18130FE
:1027C00009F045C08981813051F48A81239660E502
:1027D00070E0893311F060E070E0D1DFEDCF82303E
:1027E00021F48A8123963ADFE7CF833021F48A816E
:1027F000239698DFE1CF843041F022968111DCCF1F
:10280000CDB7DEB7E9E00C945D2F8A81239620E0F6
:1028100030E09AE0682F6053770BAB016A307105A6
:1028200060F02115310551F3EFE9FFE03197F1F741
:1028300000C0000021503109F4CF929FB001939F56
:10284000700D11249A01260F371F8991E3CFE82FCD
:10285000F0E0EE52FE4FB490282F2695269526954F
:1028600030E0F901EE53FE4FE4908770F12C082E12
:1028700002C0F594E7940A94E2F7E0FAEE24FF240C
:10288000E0F8F901EE54FE4FC490D12C082E02C09E
:10289000D594C7940A94E2F7C0FACC24DD24C0F89A
:1028A000F901EE55FE4F049110E002C01595079511
:1028B0008A95E2F701701127E114F10411F081EE1D
:1028C000CDDEC114D10411F086EEC8DE60E070E008
:1028D0008B2D55DFC114D10411F086EE23DFE114F6
:1028E000F10411F081EE1EDF0115110521F060E009
:1028F00070E08CE244DF21965FCF1F93CF93DF938C
:10290000182FA0917F03B0918003109709F449C05C
:102910001092820310928103109205031092040317
:102920001696CD91DC911797CE019A9581159F410E
:1029300008F4D07ED1E0C11101C0D0E01996ED912C
:10294000FC911A97309731F01B966D917C9180E045
:102950000995D823D11539F08CEF8C0F813A28F5E1
:102960008C2F0E94B60B1115A9F0E0917F03F09116
:102970008003808584FD0EC080917E03811551F017
:10298000808191819C01215031092F333E4710F401
:102990000E94DD0B1ADA1092800310927F031092CE
:1029A0007E03DF91CF911F9108950FDA8C2FBADE4D
:1029B000DACFCF93C6E0E0ECF1E0DF018C2F1D927F
:1029C0008A95E9F780E090E00E944C0B80E090E06F
:1029D0000E94740B10921204F8D9E2E9F2E0DF01D0
:1029E0001D92CA95E9F71092900210928F021092F0
:1029F0009102B6DCCF91089510921304DADF2FEF25
:102A000084E39CE0215080409040E1F700C000004A
:102A100088E19CE00FB6F894A895809360000FBE03
:102A200090936000FFCFAAE2B0E0E9E1F5E10C94F9
:102A3000472F8DEC91E0FC0101962091F10020835D
:102A400021E0853D9207B9F78091CE01893009F4E4
:102A50005BC0C8F4823009F4B8C0833009F487C081
:102A6000813099F18091E80083FFECC08091CD0125
:102A70009091CE019A3008F0E5C0E92FF0E0EC51DA
:102A8000FF4C0C94D32F8A3009F48EC08B3051F751
:102A90008091CD01813231F78091D1019091D201A5
:102AA000892B01F78091E800877F8093E8000E94DE
:102AB000780C81E09091CF01911101C080E080936A
:102AC00004011092130475DFCDCF8091CD01813ABE
:102AD00049F68091E800877F8093E8008091D101DA
:102AE0009091D201892B61F060E080E090E070E08D
:102AF0000E941F0C8091E8008B778093E800B2CF92
:102B000068E087ED91E0F3CF8091CD01813209F04B
:102B1000A9CF8091D1019091D2018D7F892B09F0AD
:102B2000A1CF8091E800877F8093E8008091E80042
:102B300082FF18C09091F3008091F200029731F467
:102B40008091F100813011F0863021F48091F10004
:102B5000809303018091E8008B778093E8000E94C6
:102B6000780C80CF80915E028111E0CF7BCF809185
:102B7000CD01813A09F076CF8091D1019091D201B7
:102B8000892B09F06FCF8091E800877F8093E80060
:102B90008091E80080FFFCCF809104018093F100D8
:102BA0008091E8008E77D9CF8091CD01813209F0F4
:102BB00059CF8091E800877F8093E8000E94780CCD
:102BC0008091D001809302014DCF8091CD01813A57
:102BD00009F048CF8091E800877F8093E8008091DA
:102BE000E80080FFFCCF80910201D8CF803889F0C7
:102BF000823841F58091D1018F70873018F580932C
:102C0000E9008091EB0085FB882780F91092E900AC
:102C100006C080912F02880F9091CA01892B909154
:102C2000E800977F9093E8008093F1001092F10004
:102C30008091E8008E7723C0811116C08091CF016A
:102C4000813011F18091E80083FF0AC08091E80093
:102C5000877F8093E8008091EB0080628093EB0097
:102C6000AA96E3E00C94632F823061F78091CF0144
:102C7000811589F01092E9008091E800877F8093A8
:102C8000E8000E94780CDECF81E0933009F080E00C
:102C900080932F02EFCF8091D1018F702FEF280FFB
:102CA000263080F68093E9002091EB0020FFE2CFF0
:102CB000933031F48091EB0080628093EB00DACFA7
:102CC0009091EB0090619093EB0021E030E0A9013E
:102CD00002C0440F551F8A95E2F74093EA00109214
:102CE000EA008091EB008860E8CF8111ABCF1091B2
:102CF000CF011F778091E3008078812B8093E300E0
:102D00008091E800877F8093E8000E94780C809192
:102D1000E80080FFFCCF8091E30080688093E300AF
:102D200083E0111101C082E080935E028BCF805856
:102D3000823008F087CF8091CF019091D0018C3DF7
:102D400053E0950799F583E08A838AE289834FB738
:102D5000F894DE01139620E03EE051E2E32FF0E02C
:102D600050935700849120FF03C082958F703F5F7E
:102D70008F708A30C8F0895C90E08D939D932F5FAF
:102D8000243161F74FBF8091E800877F8093E8008E
:102D90006AE270E0CE0101960E941F0C8091E8006B
:102DA0008B778093E8004ECF805DE6CF292F3327C5
:102DB0002330310509F44EC078F52130310509F48E
:102DC00088C084E790E0E2E5F2E02230310509F0C6
:102DD00039CF2091E800277F2093E8002091D3018C
:102DE0003091D4018217930708F49C0140E021152B
:102DF000310509F073C0411171C08091E80082FD76
:102E0000CDCF80915E02811549F2853039F28091F3
:102E1000E80083FFF2CFC2CF8091D1019091D2011F
:102E20002132310509F446C02232310509F00ACFBA
:102E30008430910508F006CFFC01EE0FFF1FE05E25
:102E4000FE4F0190F081E02D845E9E4FDC018C915D
:102E500090E010C09C013327823021F123303105EE
:102E600068F4232BB9F4E2E1F3E0E4918E2F90E0D3
:102E7000E2E1F3E0009709F4E5CEABCF2330310572
:102E800009F0E0CEE8EDF2E0E4918E2F90E0E8ED7D
:102E9000F2E0F0CFE2E0F3E0E4918E2F90E0E2E0A8
:102EA000F3E0E8CFE6EFF2E0E4918E2F90E0E6EF7A
:102EB000F2E0E0CF8430910508F0C4CEFC01EE0FC3
:102EC000FF1FE85DFE4F0190F081E02D89E090E06A
:102ED00080CF82E190E0E6ECF2E07BCF80915E0271
:102EE000811509F45BCF853009F458CF8091E80053
:102EF00083FD54CF8091E80082FD7FCF8091E80070
:102F000080FF75CF9091F3008091F200211531057B
:102F100019F08830910550F041E0089709F040E041
:102F20008091E8008E778093E80061CF44914093D0
:102F3000F1003196215031090196E8CF803809F02F
:102F400081CE8091E800877F8093E8008091CB015B
:102F50008093F1006DCE811175CE1091CF011230AA
:102F600008F070CE8091E800877F8093E80010938E
:102F7000CB010E94780C111521F184E080935E0250
:102F800042E061EC81E00E94F50C42E261EC84E0F9
:102F90000E94F50C42E261EC82E00E94F50C42E2F4
:102FA00060EC83E00E94F50C42E261EC85E00E9457
:102FB000F50C80915E02843051F482E0809305012B
:102FC00041CE8091E30087FDD8CF81E0D7CF81E06B
:102FD000F5CF0F93CF93DF93C7E0D4E048815981B9
:102FE0006A817B8188E090E00E94AC302881398141
:102FF0004A815B816C817D818E819F8100E20E948C
:103000002430622F83E290E00E949A30DF91CF91CA
:103010000F910895E7E0F4E085E0808311828FEF5F
:10302000828383831482CF01D4CF80910B048330B9
:1030300018F48F5F80930B0487E094E0CACF8091EF
:103040000B04811519F0815080930B0487E094E004
:10305000C0CF0F931F93CF93DF93C82F162FD42F7A
:10306000022F9091070490FF22C0E92FE695E69584
:10307000F0E0E05DFE4F8081809305049C7F9430FA
:10308000D9F46C2F712F842F0E945B08962F672F25
:10309000482F892F0E940509C09308041093090442
:1030A000D0930A04011519F087E094E092DFDF91D4
:1030B000CF911F910F910895823019F4C0910804A7
:1030C000EBCF853049F7FACFE7E0F4E0818121E0EA
:1030D00043816281885FBDCFE7E0F4E0818121E038
:1030E000438162818850B5CFE7E0F4E0628128E057
:1030F000620F08F46FEF21E043818181AACFE7E0FE
:10310000F4E0628128E0621B08F460E021E0438182
:1031100081819FCFE7E0F4E0438128E0420F08F48B
:103120004FEF21E06281818194CFE7E0F4E04381B9
:1031300028E0421B08F440E021E06281818189CFD0
:103140009091070490FF2CC0811559F18B3058F5F0
:103150008F73880F880F909107049370892B809349
:103160000704611519F087E094E033DF60910704EC
:103170006695669570E041E050E081E091E00E9444
:103180004830892B91F01092060481E0809346022A
:1031900020E040910A04609109048091080459CF0D
:1031A000089581E0D6CF8AE0D4CF81E080930604F1
:1031B0000E94C50B9093440280934302E6CF809116
:1031C0000704869586958F5F8B3008F081E061E07B
:1031D000B7CF80910704869586958A9509F48AE091
:1031E00061E0AECFAAE0B0E0E8EFF8E10C94382F50
:1031F0007C01DC0114968C91811509F417C161E002
:10320000C7010E940E108C01F7018581811541F1E3
:103210008091010490910204009711F10817190799
:10322000F9F09C013327887F9927E0E0F0E0892BB3
:1032300041F48FE0829FF001839FF00D1124E75746
:10324000FC4F84818460848311830083CF010E94BA
:10325000580F1092120461E0C7010E940E108C01F9
:103260008091F40281111BC0D70115968C918115B4
:1032700009F4A2C00034B2E51B0708F089C00115AB
:10328000E2E51E0760F40115F7E01F0741F008F0C2
:1032900064C0C801805E9109089708F063C0D70137
:1032A00015968C91811509F444C2C801975780384E
:1032B000910508F034C2003108F0B8C06EEA70E041
:1032C00080E090E00E9430108111B0C0C12CD12C60
:1032D00076010111A1C134E0332E8E010F5F1F4F23
:1032E000D801E32D1D92EA95E9F746015701FFEF5A
:1032F0008F1A9F0AAF0ABF0AC701B6010E94301099
:103300008983811509F492C0813009F005C2260134
:10331000370122E0420E511C611C711CC501B40131
:103320000E943010282E8A83811509F47FC08FEF08
:10333000820D833008F084C1C301B2010E943010B5
:103340008B83811511F0C80130DA4601570133E053
:10335000830E911CA11CB11CA2C101153FE01307F3
:1033600009F49DCF209113048091120498E0F70195
:10337000A2EEB2E001900D929A95E1F71093E90266
:103380000093E8021092EB02822B8093E10287CF38
:10339000003E42E5140750F4003C52E5150708F0E2
:1033A0007ECFC80180569245809777CF98012757E6
:1033B0003C4725303105B0F609379CE71907D1F5B0
:1033C0002091E8023091E902232B81F18115A1F0CF
:1033D00081E00E94120B8091E1020E94240F88E09C
:1033E000E2EEF2E0A9E9B2E001900D928A95E1F7F0
:1033F0008091EB028093980286E0F701A9E9B2E0A0
:1034000001900D928A95E1F7809198028093F402E1
:1034100089E992E0E7DE1092F402D70115968C91CB
:10342000811104C08091E1020E942D0F2A96E2E1F1
:103430000C94542F0A37BCE71B0709F030CF8115D5
:1034400009F4C2C0A090E802B090E902E091E10264
:10345000ED83E983BE016F5F7F4FC5010E943C0A87
:103460002C01F981F98741EAC42E42E0D42E01E013
:1034700010E022242A94D60117963C90179733FE29
:1034800053C06D907C90119712968D909C901397DD
:1034900046145704B9F41496BC91BF83232DF6014A
:1034A00046816B2F89850E94560A811559F08F81BC
:1034B0000E948505281634F4D60115969C91840146
:1034C000192B282E48145904C9F431FE17C0F601EF
:1034D000F581FF83232DD60116964C916F2F898598
:1034E0000E94560A811551F08F810E948505281689
:1034F0002CF4F60194818301192B282E30FE14C080
:10350000FFEF2F1211C00130110571F4232DD601E8
:1035100016964C9160E089850E94560A811521F02B
:10352000F60185818401182BF8E0CF0ED11C21EE25
:1035300032E02C153D0509F09ECF01301105C9F58B
:103540008D8182958F703D81832B8F7011E030319A
:1035500008F410E01295107F182BC5019A9581157B
:103560009F4108F51B29BB240A2D812F8D704A2D00
:10357000811509F44DC06AE08BEC98E00E94230BA2
:10358000282F30E02115310551F4402F6EE185EAF6
:1035900098E00E94230B282F30E0811541F0C901EB
:1035A000912B8C0106C0A11451E0B506E8F200E0B1
:1035B00010E086E0ECEEF2E0DF011D928A95E9F77B
:1035C0001093F3020093F2028091F2029091F302C1
:1035D000892B09F42BCFF7018581811539F08FEF05
:1035E0000E94120B8091EB028093EA0286E0F701C1
:1035F000ACEEB2E001900D928A95E1F78091EA027B
:103600008093F4028CEE92E0EDDD1092F4020ECF86
:1036100068E083EC98E0B2CFBFEACB16D104E104B6
:10362000F10409F403CFC701B6010E943010EFEF97
:10363000CE1ADE0AEE0AFE0A8111EECF015049CE03
:103640008BEF820D833090F54601570143E0840EE5
:10365000911CA11CB11CC301B2010E9430108B83CC
:103660008115E9F0C501B4010E9430108C838115E9
:1036700079F08B819C8181305FEF950710F0982F56
:103680008827A6E02A1671F0B7E02B1669F007D755
:1036900046015701F4E08F0E911CA11CB11C75016D
:1036A00064011ECEA9D6F4CFC8D6F2CFE4E0530110
:1036B00042012E12F4CFC301B2010E943010782EC5
:1036C00046015701F4E08F0E911CA11CB11CC701EB
:1036D000B6016D5F7F4F8F4F9F4F0E943010711466
:1036E00009F4A4CE811509F4A1CE8150990B4FEFB6
:1036F000489F9001499F300D1124472D4150550B93
:10370000240F351F2150310950F28FE99FE00197B6
:10371000F1F700C00000F6CFC80147D8C0CFF801CC
:10372000F857E730F10508F0F5C0E251FF4C0C9472
:10373000D32F6801A7E5DA1AC114B1E0DB0608F05F
:10374000E9C065EF72E08C2D0E949B11892B29F551
:103750008FE08C9DF0018D9DF00D1124E757FC4FFB
:103760008281813009F051C08091F5029091F6027A
:10377000892B99F08091F7029091F802892B69F0DA
:103780008091F9029091FA022091FB023091FC02A3
:10379000822B932B892B09F441C0F7018581811578
:1037A00071F0023AB2E51B0709F4EDC0023BE2E515
:1037B0001E0709F4CFC0013E110509F4E4C0053E1F
:1037C000110509F4C7C0809100038111F6C0D7012B
:1037D00015965C90511409F46EC10E35BCE71B07B9
:1037E00009F465C10F35ECE71E0751F00D35FCE714
:1037F0001F0709F060C180911201811509F457C1BA
:103800001092120180E079D811CE823031F6809189
:10381000F9029091FA02892B09F4BFCF2FE02C9D79
:10382000C0012D9D900D1124FC01E357FC4F208118
:103830002E7F208387579C4F0E94580FAECF83E086
:103840000E94020A8FEF92E00E948C0EEFCD80E082
:10385000F7CF8091FF02883088F088508093FF0274
:1038600091E0883008F490E08091FF0290FB80F9AD
:103870008093FF028FEF92E00E948C0E8091FF02F6
:103880008695869586950E94DF09D0CD9091FF029E
:10389000892F869586958695983140F48F5F880F9D
:1038A000880F880F9770892B8093FF028091FF0209
:1038B0008160DECF8091FF0280FF09C08E7F809300
:1038C000FF028FEF92E00E948C0E80E0DCCF8160DF
:1038D0008093FF02813071F689E0CACF8091FF02A8
:1038E0008695869586958F5F8F71843008F080E08D
:1038F000880F880F880F9091FF029770892BAECFA9
:103900008091FF0281FF03C00E94A80E8FCD0E940C
:10391000920E8CCD0337FCE71F0709F042CFD70189
:1039200015968C91811509F481CD80910003811544
:1039300019F00E94370F7ACD109213040E94C50B24
:1039400088579C4E909302038093010381E08093FB
:1039500000036CCD25EE30E02770332781E090E046
:1039600001C0880F2A95EAF72091030330910003E4
:10397000311589F0D70115963C91311539F0282B76
:103980002093030353CD21EE30E0E6CF80958223D0
:10399000809303034BCD322F3823311509F417CF11
:1039A000982F90959223909303030E945206F7015B
:1039B0008581811509F43ACD0ACFD09013040E9475
:1039C000C50B88579C4E9093020380930103D70147
:1039D00015968C91811509F4FACE8D2D8D79811172
:1039E00032C0043BB2E51B0709F4F1CEB0F5003458
:1039F000F2E51F0790F4011522E5120708F0E7CE63
:103A0000063E110509F4E3CE109212040D321105A1
:103A100069F482E08093120436C0C8018056924552
:103A20008034910508F4D3CE109212040E321105A1
:103A3000B8F50832110520F50E31110520F5C80141
:103A400004974A9730F30E94370F809113049091A6
:103A50000303892B80931304BACE09373CE713077D
:103A600050F407374CE7140708F0B1CEC801805C6A
:103A700092458097D7CF0B375CE71507A9F6A7CEFD
:103A80000A32110501F780910303811531F080910D
:103A9000120492E08927809312040E94E50E97CECB
:103AA0000C34110581F30D3282E01807EBCF81E071
:103AB00080931201BBCC80911201811143C0C801D7
:103AC00097558115914008F0D1C05801F8EFAF2209
:103AD000BB24A114B10409F0A9CC2FE0029FF0018E
:103AE0001124AF0147575C4F6A01D70115968C919D
:103AF000E357FC4F908180FB90F99083811509F486
:103B0000B5C10E94C50B9093040480930304F60191
:103B100082818F5F82838091120490911304892B9C
:103B200083834581568165857685C6010E94380B61
:103B3000D60114968C9181FF5801B0920204A09294
:103B4000010494C0380130EE631A710830901304F8
:103B500048E06416710408F05CC0980127703327B0
:103B600081E090E001C0880F2A95EAF7511409F42A
:103B70004DC0382AD7018D919C910E94FF0521E00C
:103B800030E0F90102C0EE0FFF1F8A95E2F7F887D7
:103B9000EF8320917F03309180033E832D834091FA
:103BA0008703509188035A87498796E0C92E93E08E
:103BB000D92EA12CB12C311005C0D60112968C91B2
:103BC000811119C0F601838190E02F81388582230D
:103BD0009323892B81F08085982F9770911101C0D4
:103BE00087E038E06316710408F006C1511409F447
:103BF00063C081FD63C09FEFA91AB90AAFE0CA0E86
:103C0000D11CB8E0AB16B104B1F61CC080953822C7
:103C1000B1CF51103EC0809187039091880308175F
:103C2000190781F41092880310928703109283037E
:103C300010928403109285031092860310928203DF
:103C40001092810380917F0390918003009709F483
:103C500036CFE8E06E16710408F0F2C0632D0E94C2
:103C6000840A811103C081E00E947D14F7019581CF
:103C7000911509F463C3809113048272F801E05234
:103C8000F847EB30F10508F04DC1EB50FF4C0C94B8
:103C9000D32F10938803009387030E94D10B609366
:103CA000830370938403809385039093860310921B
:103CB0008203109281035ECF82FF9DCFD6018D904B
:103CC0009C900815190519F4511409F494CFED814D
:103CD000FE81EC15FD0509F48ECFD6011D96ED9100
:103CE000FC91309721F08081811509F484CF632DF8
:103CF000C6010E94840A811509F47DCF81E0081570
:103D0000190509F080E0482E45208114910441F006
:103D1000411006C0E985FA858E169F0609F06BCF23
:103D200080E00E947D14D0928003C0927F0381E0E6
:103D300080937E038FE08A9DF0018B9DF00D11240E
:103D4000EA5FFC4F85818093050341100EC081140A
:103D5000910459F0808191819C0124503109213ACC
:103D6000310508F04FC00E94B60B8FE08A9DF0012C
:103D70008B9DF00D1124EA5FFC4FC680D780C601F1
:103D80009A9581159F4110F420EED22299249394A4
:103D9000C60101978F339E4708F0912C8FE08A9DD2
:103DA000D0018B9DB00D1124AA5FBC4F1996ED91E7
:103DB000FC911A97309731F01B966D917C9181E0C0
:103DC000099598229114A9F08FE08A9DF0018B9DAE
:103DD000F00D1124EA5FFC4F868197810E94520505
:103DE00080930403C60148E06416710470F40E94D5
:103DF000DD0B0E94E50E12C0511409F4FCCE80FDCB
:103E00005DCFF9CE0E949213B0CF0497813A91050D
:103E100058F46C2D8EEB91E00E949C0B411409F438
:103E20004ECE0E94E50E02CB0E94E50E8FE39CE988
:103E30000197F1F700C000008C2D0E942E13EECFE9
:103E4000DC012D913C910217130741F4511009C078
:103E500010927E0380E00E947D1431CE511409F44B
:103E60002ECEFC01808585FD2ACEF4CFFA01438554
:103E7000548565857685C6010E94380BD601149657
:103E80008C9181FFF3CEC6010E94400F8091010406
:103E9000909102040817190709F0E8CE1092020465
:103EA00010920104E3CE8091070480FF0BC08E7F47
:103EB0008093070487E094E08CD8109206040E9457
:103EC000F008B4CA81608093070461E08695869506
:103ED00037D9ACCA811521F07CD9A8CA8115E1F384
:103EE0006ED9A4CA811521F0F7D8A0CA8115E1F3D3
:103EF000EBD89CCA811521F002D998CA8115E1F34B
:103F0000F3D894CA811521F010D990CA8115E1F334
:103F100001D98CCA811521F092D888CA8115E1F3A4
:103F200084D884CA0737FCE71F07F9F008372CE765
:103F3000120721F19801205E32452032310518F533
:103F4000911121C00F7181E090E0AC0102C0440FDB
:103F5000551F0A95E2F78A01642F83E090E00E94E2
:103F60009A30802F0E94AB0561CA81E00E94B105A2
:103F700043E062E081E00E94330658CA82E0911576
:103F800009F4E2C1F3CF80910F04D09011042D2DDC
:103F900030E02095309550E028233523232B19F06D
:103FA0008D2180930F040B375CE7150749F49115B9
:103FB00009F43CCA8D2D0E9488050E94A50A36CAC4
:103FC000003482E5180750F50032A2E51A0760F5C3
:103FD0009801305521153240E0F1911509F45EC089
:103FE0000130ECE71E0709F457C00330FCE71F0758
:103FF00009F44CC001152CE7120709F04FC01092CC
:1040000013040E94D9143FEF44E35CE03150404078
:104010005040E1F700C000000E94060E9801205CAD
:10402000324520323105C8F6802F8F7120910F0460
:1040300030E041E050E0082E02C0440F551F0A94C2
:10404000E2F724233523232B41F2911509F4EEC91D
:10405000B4CF980185E0369527958A95E1F7822FB0
:104060008F7020910F0430E041E050E0082E02C034
:10407000440F551F0A94E2F724233523232B09F418
:10408000ACCF91119ACF10921304CBCE6FEF7FEF8C
:1040900080E090E00E94B4300E94FC14D701169694
:1040A0002D913C9121153105C9F0C9010E944D07A0
:1040B000182FD70115966C91892F82958F708830B3
:1040C00009F490C040F5843009F471C0F0F48230F6
:1040D000A0F160E0C7010E940E10A8C9F701A080FE
:1040E000B180911569F0C5010E94E40F182F682F67
:1040F000C5010E94C905B501812F0E94C90FD6CF05
:10410000C5010E94FF05182FF6CF853011F7812FCA
:104110000E947312DECF893009F4D5C08A5F8F7098
:104120008230B8F6123F09F0E0C0892F8F71611517
:1041300009F4E4C00E94BB05CCCF092F0F70903169
:1041400010F00295007F6115C9F0011569F080E259
:10415000810F883010F011110BC080911304802B57
:10416000809313040E94E50E812F0E942E13B1CF7D
:1041700080911204802B80931204F4CF812F0E942F
:104180009213011509F4A5CF80E2810F883010F059
:10419000111106C0802F0E9452060E94E50E99CF91
:1041A000009580911204802380931204F6CF892F0A
:1041B000869586958370811561F0813009F089CFED
:1041C000812F9370611102C080E090E00E94740B17
:1041D00080CF812F9370611102C080E090E00E9437
:1041E0004C0B77CF892F8370811136C0611129C0A4
:1041F000812F829586958770880F880F212F2F70C9
:10420000082E01C0220F0A94EAF7412F407114FFD3
:1042100007C04FE050E001C0440F8A95EAF740958F
:10422000969596959370923091F0842F822B9330CF
:1042300031F080911004913039F0242B82230E94B8
:10424000AB050E943D0B45CF822B842BF8CF242B4E
:10425000809110048227F3CF611589F190FFF1CF8F
:10426000812F829586958770880F880F212F2F7058
:10427000082E01C0220F0A94EAF7412F407114FF63
:1042800007C04FE050E001C0440F8A95EAF740951F
:10429000969596959370842F822B8D25923061F0A0
:1042A000842F822B933041F0842F822B8D219130EB
:1042B00019F48D2D822B842B0E94AE05C2CF823043
:1042C00008F4BFCFCDCF092F0F70611539F0802FC3
:1042D0000E94B105812F0E94150FB3CF812F0E943C
:1042E0001E0F802F0E94BB05ACCF133F51F0113F32
:1042F000A1F4892F8F71611509F41CCF0E94B105BB
:10430000E8CE80E0611531F09F7181E001C0880F37
:104310009A95EAF70E94AE05DCCE611125CF1933DC
:1043200049F4BFEFE7EEF3E0B150E040F040E1F7D1
:1043300000C00000812F0E949213CBCE07372CE7DC
:10434000120709F0F3CD81E00E94BB0511CEAEE06B
:10435000B0E0EDEAF1E20C94432F49875A876B876E
:104360007C878D879E8791111092120418861F8278
:1043700086E0FE0139968E010F5F1F4FD801019034
:104380000D928A95E1F7FD84D02EE12EF11449F0CB
:10439000FD8261E0C8010E940E1061E0C8010E9428
:1043A0000E10FD828D2D9E2D0E94F2182E96E7E0B4
:1043B0000C945F2FA6E0B0E0E0EEF1E20C94462F03
:1043C0000E94C50B8C018091650290916602801756
:1043D000910771F019821A820E94C50BBC014981B4
:1043E0005A8180E090E0B3DF10936602009365028B
:1043F0002696E4E00C94622FA6E0B0E0E2E0F2E260
:104400000C94482F9093620280936102811520E200
:10441000920730F40E947D132696E2E00C94642FFC
:1044200080EF89838A830E94C50B8160BC0149812A
:104430005A8181E091E08BDFEFCFA6E0B0E0E3E2CC
:10444000F2E20C94462F8C019093620280936102F9
:10445000011580E21807B0F4802F0E949213C80162
:10446000805E9109089728F06DE27FE00115110543
:1044700011F46EE17FE0C8010E947C052696E4E01D
:104480000C94622F80EF89838A830E94C50B816020
:10449000BC0149815A8181E090E059DFEFCFCF9391
:1044A000DF93D82FC92FA8DF8D2F9C2FC6DFDF9178
:1044B000CF9108950F931F93CF93DF938C01862F95
:1044C00065EF72E00E949B11892B91F4C091F50277
:1044D000D091F602209761F0F8018281833039F49F
:1044E000CE01DDDFCE01DBDFCE01D9DF01C0E0F799
:1044F000DF91CF911F910F9108950F931F93CF9349
:10450000DF938C01EB0165EF72E08C2F0E949B1111
:10451000892B09F057C0FE01FF27D80112968C9114
:104520001297E85EFD4F8130A9F414968C9182FDBC
:104530004EC080FF4CC082E080838091F702909152
:10454000F8020097B9F48091F5029091F602009775
:10455000C9F110C08230A1F514968C9182FD26C05D
:1045600080FD0AC083E080838091F9029091FA0275
:104570000097F1F041DF26C084E080838091FB0248
:104580009091FC020097B1F78091F5029091F602AC
:10459000009701F184DF8091F7029091F802009773
:1045A00049F78091F5029091F602E4CF85E080838F
:1045B0008091F5029091F602009721F070DFF1CF23
:1045C00086E08083DF91CF911F910F91089581E064
:1045D0008083B9CF8091F7029091F802B8CF0F9302
:1045E0001F93CF93DF938C01EB0165EF72E08C2F6B
:1045F0000E949B11892B71F4DD27C85EDD4F8881F5
:10460000F801128218828330E9F048F4813059F0C1
:10461000823081F0DF91CF911F910F910895843006
:10462000B1F08530B9F78091F5029091F6020097CC
:1046300089F306C08091F7029091F802009799F3F0
:10464000FCDEE8CF8091F9029091FA02F7CF8091D9
:10465000FB029091FC02009799F72091F5023091AE
:10466000F6028091F7029091F80221153105F9F2D6
:10467000009731F7C901E4CFA0E1B0E0E2E4F3E252
:104680000C943A2FFE01319680E1DF011D928A954C
:10469000E9F70BE010E091E5A92E93E0B92E2FEA9F
:1046A000422E512C612C712C4F0173016201B1E13A
:1046B0004B165104610471041CF080E1C82ED12C0A
:1046C000A601B501C4010E948B30AC0CBD1C0D2CA1
:1046D000000CEE08FF084C185D086E087F080150BA
:1046E000104019F76096E0E10C94562F6FEF85E2C9
:1046F00090E00E949A306FEF86E290E00E949A303C
:104700006FEF87E290E00E949A3060E088E290E0EC
:104710000E949A300E945910AFDF6AE885E290E06B
:104720000E949A3063EE86E290E00E949A3062E244
:1047300087E290E00C949A308F929F92AF92BF9252
:10474000CF92DF92EF92FF920F93CF93DF9388E0A7
:1047500090E00E9481304B015C01C7E0D4E06883A7
:104760009982AA82BB821C821D821E821F8283E2E2
:1047700090E00E947930282F30E040E050E060E087
:1047800070E080E090E000E20E9409302829392999
:104790004A295B29288339834A835B836C837D8321
:1047A0008E839F83DF91CF910F91FF90EF90DF90E9
:1047B000CF90BF90AF909F908F900895AAE0B0E007
:1047C000E4EEF3E20C943C2FFE0131968AE0DF0127
:1047D0001D928A95E9F79BE3A92E91E0B92E8F01EE
:1047E0003F01EE24E394F12C3FE4C32E31E0D32EBD
:1047F000F50181915F018F3F09F444C0F894E82FDF
:10480000E295EF70F0E021A18F70A70102C0440F84
:10481000551F8A95E2F7CA01922F982B91A392A176
:104820008095892382A3789400C0E0E4F1E021E040
:1048300030E0812C912C41914F3F79F0A42FA2952B
:10484000AF70A05EB0E08C9190E04F7002C0959583
:1048500087954A95E2F780FF3BC080E090E0882A88
:10486000992A220F331FCE16DF0629F7F501829110
:104870008F3F11F00E94410850EA5A95F1F7D80194
:104880008D929C920E5F1F4FB0E4AB16B1E0BB0659
:1048900009F0AECF4AE050E0B30180E292E00E941E
:1048A0005530892BB9F08AE0F301A0E2B2E0019023
:1048B0000D928A95E1F781E08093C8010E94C50BB3
:1048C0009093C7018093C6012A96EEE00C94582F6E
:1048D000C901C5CF8091C8018115B1F30091C6010E
:1048E0001091C7010E94C50B801B910B059760F3C7
:1048F0004AE050E060E272E082E592E00E945530CA
:10490000892B49F08AE0E0E2F2E0A2E5B2E0019012
:104910000D928A95E1F71092C801D6CFCDB7DEB7D8
:10492000AD970FB6F894DEBF0FBECDBF85B78068D8
:1049300085BF85B7806885BF84B7877F84BF0FB682
:10494000F894A8958091600088618093600010922F
:1049500060000FBE80E890E00FB6F894809361008D
:10496000909361000FBE81E0809305018FE79DE089
:104970009093BD018093BC010E94240A0E94DE1026
:104980000E945D110E94C80C0E94250D8091E200DA
:1049900084608093E200789480915E02811599F0A2
:1049A0008091E9001091EC008F70179511271795F1
:1049B000182B1092E9008091E80083FD0E941315E6
:1049C0001F701093E90082E084BD93E095BD9AEFDB
:1049D00097BD80936E000E944010811101C086DE59
:1049E0000BE311E0D8018D918D018F3F11F00E94F2
:1049F0004108B1E000341B07A9F700E411E0F80119
:104A000081918F018F3F11F00E944108F1E00F3436
:104A10001F07A9F78AE0E2E5F2E0DF01282F1D92E7
:104A20002A95E9F7E0E2F2E0DF011D928A95E9F7C5
:104A300080E090E00E948630833E9E4F21F40E94E9
:104A4000401081112FC063EE7EEF80E090E00E9465
:104A5000B43060E082E090E00E949A3081E0809380
:104A6000100461E083E090E00E949A3060E074E11D
:104A700084E090E00E94B4301982CE0101960E9439
:104A80008C0E0E940A1832DE40E050E0BA018FE03E
:104A900090E00E94AC3040E050E0BA0183E190E049
:104AA0000E94AC3082E090E00E9479308093300226
:104AB00084E090E00E9486309093600280935F02D1
:104AC0007DDEEFEFF6E721E0E150F0402040E1F736
:104AD00000C0000073DE8091520280FF08C06FEFBB
:104AE0007FEF80E090E00E94B4300E94060E83E0E9
:104AF00090E00E9479300E94AB05279A2F988AE0B7
:104B00008093800089E1809381008FEF9FEF9093E5
:104B10008700809386000E94790F8091FF0281FFB9
:104B20000BC010922C0210922B0210922A0280913C
:104B30006F00816080936F000E94790F80912D0239
:104B400081111EC087E094E0F7DD80910704843076
:104B500028F40E940A1887E094E0EEDD0E94E20843
:104B6000109206040E94770A8091070480FF05C016
:104B700060E0869586950E94A01881E080932D02C2
:104B800086E091E0909368028093670280915E02D4
:104B9000853069F480915E02853009F4B0C01092CE
:104BA00013040E94D9140E94790F0E943D0B06DE67
:104BB00061E3A62E62E0B62E02E512E0D801F5010F
:104BC000219131918D919D914BE352E04E175F07FA
:104BD00009F4CDC02817390799F38091300281FF7D
:104BE0004DC08CE597E09F938F930E9449050F90ED
:104BF0000F9092E5C92E92E0D92EE12CF12C27E5F9
:104C0000822E27E0922E34E5632E37E0732E4EE499
:104C1000442E47E0542E5CE4252E57E0352EFF92BB
:104C2000EF929F928F920E9449057F926F920E940D
:104C30004905D6018C911196BC91BDA7E2E0CE0E3C
:104C4000D11C0E949B058BA78DA50E949B05FBA5EF
:104C5000FF938F935F924F920E9449053F922F924C
:104C60000E9449052FEFE21AF20A0FB6F894DEBF50
:104C70000FBECDBF55E0E516F10489F6A2E56A2E18
:104C8000A2E07A2E512CD301ED90FD903D01F5016B
:104C9000819091905F018E149F0451F18E249F2486
:104CA000412CCC24C394D12CC4018C219D21892B6F
:104CB000B1F049825A820E94C50B9C838B83F1E03C
:104CC000FD8391E097012C213D21232B09F490E0F5
:104CD0009E8349815A816B817C818D8138DB43942D
:104CE000CC0CDD1C2FE04212DFCFF501F292E292F4
:104CF000539435E05312C7CF0E94D10B3DC0809131
:104D00005E02843039F180E00E94020A10922E0285
:104D100048E150E080E40FB6F894A8954093600015
:104D20000FBE8093600083B7817F846083BF83B7A9
:104D3000816083BF7894889583B78E7F83BF0FB6D9
:104D4000F894A8958091600088618093600010922B
:104D500060000FBE33DDE2E5F2E081919191892B95
:104D600009F00FC692E0EC35F907B9F713CF281711
:104D7000390709F032CF1EDBE0908103F090820307
:104D8000E114F10491F180903F0290904002A090D4
:104D90004102B09042020E94D10B681979098A0938
:104DA0009B0980903B0290903C02A0903D02B09005
:104DB0003E02681579058A059B05B8F0C7010E9477
:104DC0007D13109282031092810310923F02109281
:104DD0004002109241021092420210923B02109245
:104DE0003C0210923D0210923E02C0900104D0900D
:104DF0000204C114D10411F1E0900304F090040402
:104E00000E94C50B8E199F09893C9105B8F0960147
:104E1000332748EFC422DD2480E090E0CD2841F420
:104E20004FE0429FC001439F900D112487579C4F34
:104E3000DC0114962C9122FF0E94580F80910003F0
:104E4000811569F00E94C50B209101033091020386
:104E5000821B930B8F3F9F4710F40E94370F809166
:104E600006048115D9F180910504E0910704E695C7
:104E7000E695E81BE0934502823009F041C1F0E07D
:104E8000EA58F84FE491EE2EF12CF2E2CF2EF9E041
:104E9000DF2E80914602811561F0109246020E9439
:104EA000C50B9093440280934302109248021092E3
:104EB00047020E94C50B2091430230914402821B9D
:104EC000930B8F3F9F4750F42E0D3F1D30934402AC
:104ED0002093430283E492E0F601099586E0E2E93B
:104EE000F2E0DE01119601900D928A95E1F7909023
:104EF0009302B0909402F0909502A0909602E090F8
:104F000097021092940210929502109296021092BB
:104F100097028F2D8B29811509F441C0C0904B0257
:104F2000D0904C020E94C50B9C012C193D09909118
:104F30009002911509F420C52531310580F19F3F7C
:104F400019F09F5F90939002B11459F00E94CD0A1E
:104F500091E01B140CF09FEF899F802D112480930A
:104F60009402F11459F00E94CD0A91E01F140CF044
:104F70009FEF899F802D1124809395028091940248
:104F8000811569F0D0909502D11449F00E94BF0AB2
:104F9000809394028D2D0E94BF0A809395028A2DE2
:104FA0008E29811509F441C0C0904902D0904A026F
:104FB0000E94C50B9C012C193D0990918F029115FF
:104FC00009F4D5C42135310580F19F3F19F09F5F69
:104FD00090938F02A11459F00E94ED0A91E01A14E7
:104FE0000CF09FEF899F802D112480939602E1148D
:104FF00059F00E94ED0A91E01E140CF09FEF899F7A
:10500000802D11248093970280919602811569F07A
:10501000D0909702D11449F00E94BF0A8093960263
:105020008D2D0E94BF0A809397028091930298125F
:1050300019C080919402811511F08B1113C0209139
:105040009502211511F02F110DC090919702911525
:1050500011F09E1107C030919602311103C0822BCE
:10506000892B81110E94B01186E0FE013196A2E9E0
:10507000B2E001900D928A95E1F70E943D0B90916C
:105080004D02891721F080934D020E94D10B80912F
:105090005E02843009F07ACD83E08093E90080914C
:1050A000E80082FF73CD8091E80090E085FF05C0A5
:1050B0000E94970C8115D9F191E08091E8008B77DF
:1050C0008093E800911509F461CDE0906302F090BF
:1050D0006402E981E114F10409F448C0EE3F09F0EB
:1050E00068C08A81833020F08550833008F061C029
:1050F000EA81EE3008F05DC0F0E0E050FF4C53C7AD
:1051000060EDE62E67E0F62E7AE5C72E78E0D72E22
:10511000853009F0BECEE695F0E0ED58F84FE49109
:10512000EE2EF12CEAE3CE2EE9E0DE2EB2CE50E2F6
:10513000C52ED12C9E012F5F3F4F79018091E80051
:1051400085FD0AC08091E8008B778093E8000E947B
:10515000970C811599F3B0CF8091F100D7018D9311
:105160007D01B1E0CB1AD10849F7A6CFE43148F46C
:10517000E11551F0E150E33138F4F0E0E25FFE4C2C
:1051800012C7EE3F09F4B4CF8FEF898312C01A82A1
:1051900089E08B830EC08A81823081F08330B1F048
:1051A000813091F70E94D10B14D76B837C838D8360
:1051B0009E83CE0101960E94E70CE8CC88E290E045
:1051C00098D71B821C821D828E83F3CF80915C0254
:1051D00090915D02892B69F3FE013196D8018C9183
:1051E00011969C910E5F1F4F928383833296B2E09B
:1051F0000C351B0799F7DDCF8A81823029F66B8148
:105200007C818D819E81E5D688E290E093D7D1CFD5
:105210004C816B818A810E949A0F98278927982751
:105220009E838D83C6CF2D813E813227232732274F
:105230004C816B818A810E94BE0EBBCF0E945910A7
:10524000B8CF8A818930E9F08A3049F18A81823881
:1052500009F449C068F58038A1F1813809F0A9CF77
:1052600060E08B810E94A0189B81809107049111BE
:1052700031C08E7F80930704109206040E94F008CC
:1052800098CF2B8130E0C901880F991F820F931F9F
:105290006FEF70E03FD6862F0E94020AD7CF8B8136
:1052A000811103C00E94A80ED1CF0E94920ECECFD2
:1052B000833809F07ECF20E040910A046C818B8115
:1052C00006C020E04B8160910904809108040E948F
:1052D00029186FCF81608093070460E086958695DA
:1052E0000E94A01866CF8B8180930B0462CF8A81C5
:1052F000893089F08A30C9F0823859F1D8F4803881
:1053000019F1813809F055CF8091070480FF1FC043
:10531000869586953ECF8091FF02869586958695E7
:10532000E5E58E9FC001112434CF8091FF02869560
:1053300081702FCF833809F03CCF809108048B8394
:10534000809109048C8335CF80910A0422CF80E0BC
:1053500020CF80910B041DCF8FEF92E00E948C0E26
:105360000E94E20887E094E00E94E91722CF80E1E2
:105370008A831FCF1A828FEA0CCF8C818D3108F07F
:1053800018CF8A809B80982489249824A12CB12C42
:105390008E010F5F1F4F7801E80EF11C0E151F05DF
:1053A00009F407CF80E0FFEA8F169104A104B1044D
:1053B00020F4C4018F5A9C4F9CD6D80114968C932C
:1053C0000F5F1F4FBFEF8B1A9B0AAB0ABB0AE6CFDA
:1053D00080915C0290915D02892B09F4EACE8C8168
:1053E0008D3108F0E6CE882E912CA12CB12CCA80EC
:1053F000DB80DC24CD24DC24E12CF12C8E010F5F3A
:105400001F4F412C512C3201481459046A047B046B
:1054100008F0CFCEEFEACE16D104E104F10438F45F
:10542000D80114966C91C6018F5A9C4F83D6BFEF5A
:105430004B1A5B0A6B0A7B0AEFEFCE1ADE0AEE0A02
:10544000FE0A0F5F1F4FE0CF17D9B3CE84E090CF95
:105450008C818D3108F0ADCE882E912CA12CB12CF1
:10546000CA80DB80DC24CD24DC24E12CF12C412C0F
:10547000512C32018E010B5F1F4F481459046A04EE
:105480007B0408F096CE80E0F8E5CF16F2E0DF0668
:10549000E104F10418F4C60189962BD6D8018D9346
:1054A0008D01BFEF4B1A5B0A6B0A7B0AEFEFCE1A36
:1054B000DE0AEE0AFE0AE1CF2C81022F10E02D3128
:1054C00008F077CE8A819B819827892798272C011D
:1054D000612C712C8835F2E09F0708F06ACE822E8D
:1054E000912CA12CB12C48E552E060E070E0441909
:1054F000550966097709421751056105710508F4D8
:1055000058CE20915C0230915D02232B09F03EC001
:105510001C0129E2220E311C80FBEE24FF24E0F85E
:1055200080FF0BC08896E5D59D818927982789271C
:1055300081159C4711F48FEF8D83D501C401840D33
:10554000951DA61DB71D80FF19C0680141E0C41A52
:10555000D108CE0105968C0D9D1D9CA78BA7C1017E
:10556000800F911FC6D5ABA5BCA59C9181159C470A
:1055700021F48FEFEBA5FCA580838601FE01319617
:10558000EE0DFF1D2FEFE016F10638F08E010F5FD4
:105590001F4FC12CD12C760125C0948185818115A6
:1055A0009C4711F42483258342E0E40EF11C3296DB
:1055B000EACF58E5451652E055066104710430F40F
:1055C000D80114966C91C2018996B4D5BFEFCB1A5D
:1055D000DB0AEB0AFB0AEFEF4E1A5E0A6E0A7E0A3E
:1055E0000F5F1F4FC814D904EA04FB0410F3E1CD88
:1055F00080915C0290915D02892B09F4DACDCE0195
:1056000001960E94E70CFFEF21EE34E0F1502040BC
:105610003040E1F700C0000068CA88E0E3E1F1E053
:10562000DE01919601900D928A95E1F7FE01329686
:105630008FE1DF011D928A95E9F786E0898388E092
:105640007F96DE01159601900D928A95E1F7B1CD16
:105650008CE2898381E08A831B821C82AACD8B81A4
:105660009C81092E000CAA0BBB0B25E0880F991F0B
:10567000AA1FBB1F2A95D1F7AC01BD01405E5F4F49
:105680006F4F7F4F481759076A077B0708F491CD82
:105690008C32E1E09E07A105B10508F08ACD4D32BC
:1056A000F1E05F076105710520F04CE251E060E038
:1056B00070E0481B590BBC016758784FCE0101962A
:1056C000DED477CD4AE150E06FEF70E0CE0107966F
:1056D000F9D480915C028983EA821B821C8281E07A
:1056E0008D8372CD81E090E0909364028093630299
:1056F00082E390E090935102809350020E94C50B88
:1057000090934F0280934E0254CDE114F10481F145
:10571000D0905202C090540200914E0210914F025C
:105720000E94C50B801B910B8536910540F1C1FE8F
:1057300026C0D0FE24C00E94C50B90934F028093D8
:105740004E02809150029091510201979093510224
:1057500080935002892B61F41092640210926302CC
:1057600081E090E090935D0280935C02E12CF12C4B
:1057700080915C028983EA82809150020ACD82E3A3
:1057800090E09093510280935002F2CF10925D020C
:1057900010925C020ECD40E250E06FEF70E0CE015F
:1057A000019690D406CDEB81E93008F002CDF0E00F
:1057B000EF5DFE4CF8C3FE0132968EE1DF011D92D3
:1057C0008A95E9F788E089838B838C8383E088A3BB
:1057D000F0CC8C819AE0F92E8E010F5D1F4FF801FD
:1057E0002F2D11922A95E9F7B8010E949B11898308
:1057F000F801DE01129601900D92FA94E1F7D9CCEE
:105800001C818AE0FE013596DE01919601900D9291
:105810008A95E1F789A19AA10E94170A9AA389A300
:105820008BA19CA10E94170A9CA38BA38DA19EA172
:105830000E94170A9EA38DA38FA198A50E94170A04
:1058400098A78FA38FEF183060F43AE0139FB00150
:1058500011246F577D4F4AE050E0CE01819688D4E5
:1058600080E089830E94240AA4CC2C816AE0CE01C6
:105870008196DC01E62F1D92EA95E9F7283080F445
:10588000629FB00111246F527D4F4AE050E021D455
:1058900080E089838AE0FE01B196DE011296D3CEC4
:1058A0008FEFF7CF1C818AE0FE013596DE019196DD
:1058B00001900D928A95E1F78BA19CA10E94170A95
:1058C0009CA38BA38FEF183060F4FAE01F9FB00108
:1058D00011246F527D4F4AE050E0CE01819648D4AA
:1058E00080E089830E94DE1064CC2C8166E0CE01CA
:1058F0008196DC01E62F1D92EA95E9F7283060F4E5
:10590000629FB00111246F5D7C4F46E050E0E1D30F
:1059100080E0898386E0BFCF8FEFFBCF1C8186E0DC
:10592000FE013596DE01919601900D928A95E1F780
:1059300089A19AA10E94170A9AA389A38BA19CA16D
:105940000E94170A9CA38BA38FEF183060F4F6E037
:105950001F9FB00111246F5D7C4F46E050E0CE01E7
:10596000819606D480E089830E945D1122CC2B3081
:10597000310508F02CCB59CB2B30310508F0E1CAAA
:105980000ECB80912F02811509F404C9A0E1A9BDB5
:10599000B2E1B9BD09B400FEFDCF8091D8008F7D82
:1059A0008093D8008091E00082608093E000809135
:1059B000E00081FDFCCF109213040E94D914EAC8C4
:1059C0001F920F920FB60F9211242F933F934F9374
:1059D0005F936F937F938F939F93AF93BF93EF9357
:1059E000FF93809100018230A1F08F5F80930001CE
:1059F000FF91EF91BF91AF919F918F917F916F91A7
:105A00005F914F913F912F910F900FBE0F901F907C
:105A1000189581E08093000180912B0290912C02D7
:105A2000019660ED72E076D290932C0280932B0267
:105A300065E070E06FD267FD6FE780912A028230E7
:105A400069F5603429F480916F008E7F80936F0038
:105A5000E62FF0E0E453FA4F2491A0918600B09134
:105A6000870030E0BDD22FEF30E040E050E079D247
:105A7000C90163E070E04ED28091FF028695869561
:105A80008695282F269FC001279F900D11240E94E4
:105A9000630990938D0080938C00AACF8130C1F66A
:105AA0006F37D0CF1F921FB61F9211248F939F93F1
:105AB000AF93BF9380912E02811113C08091DF01BB
:105AC0009091E001A091E101B091E2014196A11D08
:105AD000B11D8093DF019093E001A093E101B093A9
:105AE000E201BF91AF919F918F911F901FBE1F90B8
:105AF000189578941F921FB61F9211248F939F932D
:105B0000AF93BF938091DF019091E001A091E101FB
:105B1000B091E2010196A11DB11D8093DF01909328
:105B2000E001A093E101B093E201BF91AF919F9199
:105B30008F911F901FBE1F9018951F920F920FB646
:105B40000F9211242F933F934F935F936F937F9303
:105B50008F939F93AF93BF93EF93FF938091E10057
:105B600082FF14C08091E20082FF10C08091E100AA
:105B70008B7F8093E1002091C9012F5F822F62E328
:105B8000BDD1911509F4DCC02093C9018091DA00E0
:105B900080FF2CC08091D80080FF28C08091DA005F
:105BA0008E7F8093DA008091D90080FFFEC080E173
:105BB00089BD82E189BD09B400FEFDCF81E08093FB
:105BC0005E0286E193E09F938F930E944905809146
:105BD000CC010F900F90811109C00E94C80C0E9447
:105BE000250D8091E20084608093E2008091E100C5
:105BF00080FF22C08091E20080FF1EC08091E20001
:105C00008E7F8093E2008091E20080618093E200C9
:105C10008091D80080628093D80019BC85E0809381
:105C20005E028EE193E09F938F930E94490583E08B
:105C3000809305010F900F908091E10084FF37C0A1
:105C40008091E20084FF33C080E189BD82E189BD9B
:105C500009B400FEFDCF8091D8008F7D8093D800DD
:105C60008091E1008F7E8093E1008091E2008F7E41
:105C70008093E2008091E20081608093E200809155
:105C8000CB01811509F49FC084E080935E0282E21B
:105C900093E09F938F930E94490580915E020F903D
:105CA0000F90843009F097C082E0809305018091C5
:105CB000E10083FF34C08091E20083FF30C0809117
:105CC000E100877F8093E10082E080935E02109282
:105CD000CB018091E1008E7F8093E1008091E20012
:105CE0008E7F8093E2008091E20080618093E200E9
:105CF00042E060E080E00E94F50C8091F000886056
:105D00008093F00086E293E09F938F930E94490571
:105D100081E080930501809304010F900F90FF9123
:105D2000EF91BF91AF919F918F917F916F915F9113
:105D30004F913F912F910F900FBE0F901F9018958C
:105D40001092C9018091D601811509F41FCF80916D
:105D50005E028430B9F49091E9008091EC009F706C
:105D6000879588278795892B95E09093E9009091F6
:105D7000EB0090FF04C09091EE0097FD08C08F707B
:105D80008093E9001092D60101CF1092F10090911A
:105D9000E80095FDFACF9091E80090FFF0CF909148
:105DA000E8009E779093E800EACF19BC10925E025B
:105DB0008AE193E09F938F930E9449051092CC0152
:105DC0000F900F9013CF8091E30087FF02C083E014
:105DD0005CCF81E05ACF81E068CF1F920F920FB65F
:105DE0000F921124EF92FF920F931F932F933F93E3
:105DF0004F935F936F937F938F939F93AF93BF93D3
:105E0000CF93EF93FF9309EE10E0F8018081C091EA
:105E1000EC008F70C795CC27C795C82B108280EFF8
:105E2000E82EF12CF7018081877F808378940E948F
:105E30001315F8011082F701808188608083CF708C
:105E4000F801C083FF91EF91CF91BF91AF919F91E6
:105E50008F917F916F915F914F913F912F911F9102
:105E60000F91FF90EF900F900FBE0F901F9018951D
:105E70002F923F924F925F926F927F928F929F925A
:105E8000AF92BF92CF92DF92EF92FF920F931F9348
:105E9000CF93DF93CDB7DEB7CA1BDB0B0FB6F894F9
:105EA000DEBF0FBECDBF09942A88398848885F8439
:105EB0006E847D848C849B84AA84B984C884DF80AA
:105EC000EE80FD800C811B81AA81B981CE0FD11D8E
:105ED0000FB6F894DEBF0FBECDBFED010895DB0114
:105EE0008F939F938CD0BF91AF91A29F800D911DF6
:105EF000A39F900DB29F900D11240895992778E0EB
:105F0000880F991F961708F0961B881F7A95C9F776
:105F100080950895AA1BBB1B51E107C0AA1FBB1F98
:105F2000A617B70710F0A61BB70B881F991F5A9525
:105F3000A9F780959095BC01CD01089597FB072E98
:105F400016F4009406D077FD08D0E4DF07FC05D0F6
:105F50003EF4909581959F4F0895709561957F4F80
:105F60000895A1E21A2EAA1BBB1BFD010DC0AA1F9A
:105F7000BB1FEE1FFF1FA217B307E407F50720F0B2
:105F8000A21BB30BE40BF50B661F771F881F991F2D
:105F90001A9469F760957095809590959B01AC0176
:105FA000BD01CF010895EE0FFF1F0590F491E02D84
:105FB0000994082E817006940694811D0694811D13
:105FC0000694811D0694811D0694811D0694801DF2
:105FD00008956927962769277827872778270895BE
:105FE000A29FB001B39FC001A39F700D811D11241A
:105FF000911DB29F700D811D1124911D0895F0DF38
:10600000A59F900DB49F900DA49F800D911D11240C
:106010000895002E083090F0982F872F762F652F47
:10602000542F432F322F22270850F4CF220F331F33
:10603000441F551F661F771F881F991F0A95B2F7C7
:10604000002D089597FD1094002E083098F0085008
:10605000232F342F452F562F672F782F892F912DDF
:10606000F4CF1594979587957795679557954795AC
:10607000379527950A95AAF71124002D0895FB015D
:10608000DC0102C005900D9241505040D8F70895B0
:10609000FC014150504030F001900616D1F7319785
:1060A000CF010895882799270895FB01DC0104C0DA
:1060B0008D910190801921F441505040C8F7881B00
:1060C000990B0895DC0101C06D9341505040E0F7F9
:1060D0000895DC01CB01FC01F999FECF06C0F2BDA9
:1060E000E1BDF89A319600B40D9241505040B8F796
:1060F0000895F999FECF92BD81BDF89A992780B590
:106100000895A6E1B0E044E050E0E5CFA8E1B0E0BA
:1061100042E050E0E0CFDC01A40FB51F41505040F9
:1061200040F0CB01840F951F2E9105D04150504077
:10613000D8F70895262FF999FECF92BD81BDF89A20
:10614000019700B4021639F01FBA20BD0FB6F894BB
:10615000FA9AF99A0FBE08950396272FECDFEADF2B
:10616000252FE9DF242FE7CF0196272FE4DFE2CFA9
:10617000DC01CB0102C02D9105D041505040D8F731
:106180000895262FF999FECF1FBA92BD81BD20BD7B
:106190000FB6F894FA9AF99A0FBE01960895F894FA
:1061A000FFCF7F12841286128B129B129B129B12BE
:1061B0009B129B129B129B129B128D129112941296
:1061C0009912A912AF12B312F6151C1622161C163C
:1061D00022167516971622169E17AB171F1C271C22
:1061E0005A1C291C461C6E1C801C531F6A1F6E1FE4
:1061F000721F761F7A1F7E1F821F861F8A1F8E1FA7
:106200000D2B282B2F2BD928D928622B722B852BCD
:10621000C62BCB2BD928D928D928D32BC728CB28B4
:10622000FC28082913291E2921297729AC29C428EB
:10623000F82AB729BA29BD29E829242A262A282A92
:106240005C2ADB2BE92B002CD928D928352C522CA1
:04625000752C8E2CEF
:10625400010100000100C20B6C0E1E0C820E870EA1
:10626400630E01DC0B71F924BD07B40044227B15D5
:106274005E013C01C100AC0064027D029D02B602D5
:10628400000102020205050505050530336736667F
:10629400F6F5F4F1C695939291909496973435E27D
:1062A40000E900EA00B500B600B700CD008301CCD8
:1062B400008A01920194012102230224022502266C
:1062C4000227022A02B300B4006F0070009F01CBC2
:1062D400019F02A002E200E900EA00B500B600B79F
:1062E40000CD008301CC008A019201940121022394
:1062F4000224022502260227022A02B300B4006FF8
:0C6304000070009F01CB019F02A002006E
:00000001FF
